:020000040000FA
:0400000000002229B1
:08000800A000030E8312A10009
:100010000A08A2000408A3000B1C1E2805080B10E8
:10002000BA01BB01BC014608B20085191B28043087
:10003000B10005101E280130B10005148C1CC22827
:100040008C1000308A003108820757282A282C2873
:100050007D282E283D302F2840302F284330840023
:100060000008BC07031C3928BB0F3928BA0A03193A
:100070004628840A0008BB07031C4128BA0A031952
:100080004628840A0008BA07031C4E28BA01BB019F
:10009000BC01B10A3108053A0319B10100308A00E8
:1000A0003108820757285A286C287D288128C801E2
:1000B000C901B8283209AC003A08071A6528C121DD
:1000C000A8003A0AC121A900EF20CB2032082D0751
:1000D000C6002E08C70094283509AC003A08071A54
:1000E0007728C922A8003A0AC922A900EF20CB200C
:1000F0002D09C6002E09C70094283508C600C7017F
:1001000094283208AC003A08071A8C28C922A800A3
:100110003A0AC922A900EF20CB2032092D07FF3A65
:10012000C6002E09C7009428C801C9013808031069
:100130004618C807C80CC90CC618C807C80CC90C93
:100140004619C807C80CC90CC619C807C80CC90C81
:10015000461AC807C80CC90CC61AC807C80CC90C6F
:10016000461BC807C80CC90CC61BC807C80CC90C5D
:10017000490D9516031C9512490D1516031C1512F1
:100180004808930022088A0023088400210E830077
:10019000A00E200E0900AD01AE0103102C18AD0712
:1001A000AD0CAE0CAC18AD07AD0CAE0C2C19AD07F8
:1001B000AD0CAE0CAC19AD07AD0CAE0C2C1AAD07E6
:1001C000AD0CAE0CAC1AAD07AD0CAE0C2C1BAD07D4
:1001D000AD0CAE0CAC1BAD07AD0CAE0C0800280886
:1001E000A902AA01AB01290803103B18AA07AA0C0F
:1001F000AB0CBB18AA07AA0CAB0C3B19AA07AA0C9C
:10020000AB0CBB19AA07AA0CAB0C3B1AAA07AA0C89
:10021000AB0CBB1AAA07AA0CAB0C3B1BAA07AA0C77
:10022000AB0CBB1BAA07AA0CAB0C28082A070800BA
:100230000630A400A40B1A299F149F181D291E081C
:10024000B000080087010730990091010430920046
:100250009301831602308C00F630910020309F000D
:10026000FF3092001F3087003E3085000830960036
:10027000831200308C00C8308B000C309500B30125
:10028000B401B501B6018030B700FF30B800B1014C
:10029000B901BC01BB01BA01BD01BE01BF01C00172
:1002A000C101C201C301C401C501C601C701C80122
:1002B000C9010730AF000510B201AF0A01308A0052
:1002C0002F08073982076B29822999299E29B52988
:1002D000BC29AF0A5D2905309F0018213707031C90
:1002E0007529A700A71B7F307829A700A71F80309A
:1002F000803EB300A600D123BF00D824BE00DF2576
:10030000BD005D2909309F0018213707031C8C2987
:10031000A700A71B7F308F29A700A71F8030803E32
:10032000B400A600D123C200D824C100DF25C0003C
:100330005D2911309F001821B5005D2915309F00FF
:1003400018213707031CA829A700A71B7F30AB295A
:10035000A700A71F8030803EB600A600D123C500AD
:10036000D824C400DF25C3005D2919309F0018215F
:100370008030FF3AB7005D291D309F001821B8007A
:100380005D29A50001308A002508C93E03188A0AA4
:1003900082000034013403340534073409340B344B
:1003A0000D340E3410341234143416341734193416
:1003B0001B341D341E342034223423342534273496
:1003C00029342A342C342D342F343134323434341B
:1003D0003634373439343A343C343D343F344134A4
:1003E000423444344534473448344A344B344C3432
:1003F0004E344F34513452345434553457345834C5
:1004000059345B345C345D345F346034623463345B
:10041000643466346734683469346B346C346D34F6
:100420006F34703471347234743475347634773494
:1004300079347A347B347C347D347E348034813436
:1004400082348334843485348734883489348A34DC
:100450008B348C348D348E348F3490349234933486
:100460009434953496349734983499349A349B3430
:100470009C349D349E349F34A034A134A234A334E0
:10048000A434A534A634A734A834A934AA34AA3491
:10049000AB34AC34AD34AE34AF34B034B134B23448
:1004A000B334B334B434B534B634B734B834B934FF
:1004B000B934BA34BB34BC34BD34BE34BE34BF34BA
:1004C000C034C134C234C234C334C434C534C63475
:1004D000C634C734C834C934C934CA34CB34CC3434
:1004E000CC34CD34CE34CE34CF34D034D134D134F6
:1004F000D234D334D334D434D534D534D634D734B9
:10050000D834D834D934DA34DA34DB34DB34DC347C
:10051000DD34DD34DE34DF34DF34E034E134E13443
:10052000E234E234E334E434E434E534E534E6340C
:10053000E734E734E834E834E934E934EA34EB34D6
:10054000EB34EC34EC34ED34ED34EE34EE34EF34A3
:10055000EF34F034F034F134F234F234F334F33471
:10056000F434F434F534F534F634F634F734F7343F
:10057000F834F834F934F934F934FA34FA34FB3411
:10058000FB34FC34FC34FD34FD34FE34FE34FF34E3
:10059000FF34A50002308A002508D13E03188A0ADC
:1005A0008200003407340E3414341B3421342834D0
:1005B0002E34343439343F34443449344F34533492
:1005C00058345D34623466346A346E34723476344E
:1005D0007A347E348234853489348C348F34923446
:1005E000953498349B349E34A134A334A634A83473
:1005F000AB34AD34B034B234B434B634B834BA34C5
:10060000BC34BE34C034C234C334C534C734C83437
:10061000CA34CB34CD34CE34D034D134D234D334C4
:10062000D534D634D734D834D934DA34DB34DC3466
:10063000DD34DE34DF34E034E134E234E334E43416
:10064000E434E534E634E734E734E834E934E934D3
:10065000EA34EA34EB34EC34EC34ED34ED34EE349B
:10066000EE34EF34EF34F034F034F134F134F1346B
:10067000F234F234F334F334F334F434F434F43441
:10068000F534F534F534F534F634F634F634F7341D
:10069000F734F734F734F734F834F834F834F834FE
:1006A000F934F934F934F934F934F934FA34FA34E0
:1006B000FA34FA34FA34FA34FB34FB34FB34FB34C6
:1006C000FB34FB34FB34FB34FC34FC34FC34FC34AE
:1006D000FC34FC34FC34FC34FC34FC34FD34FD3498
:1006E000FD34FD34FD34FD34FD34FD34FD34FD3482
:1006F000FD34FD34FD34FD34FE34FE34FE34FE346E
:10070000FE34FE34FE34FE34FE34FE34FE34FE3459
:10071000FE34FE34FE34FE34FE34FE34FE34FE3449
:10072000FE34FE34FE34FE34FE34FF34FF34FF3436
:10073000FF34FF34FF34FF34FF34FF34FF34FF3421
:10074000FF34FF34FF34FF34FF34FF34FF34FF3411
:10075000FF34FF34FF34FF34FF34FF34FF34FF3401
:10076000FF34FF34FF34FF34FF34FF34FF34FF34F1
:10077000FF34FF34FF34FF34FF34FF34FF34FF34E1
:10078000FF34FF34FF34FF34FF34FF34FF34FF34D1
:10079000FF34FF34FF34FF34FF34FF34FF34FF34C1
:1007A000FF3403308A002608D83E03188A0A8200E4
:1007B0000634063405340534043404340434043473
:1007C0000334033403340334033402340234023474
:1007D000023402340234013401340134013401346E
:1007E0000134013401340134003400340034003465
:1007F0000034003400340034003400340034003459
:100800000034003400340034003400340034003448
:100810000034003400340034003400340034003438
:100820000034003400340034003400340034003428
:100830000034003400340034003400340034003418
:100840000034003400340034003400340034003408
:1008500000340034003400340034003400340034F8
:1008600000340034003400340034003400340034E8
:1008700000340034003400340034003400340034D8
:1008800000340034003400340034003400340034C8
:1008900000340034003400340034003400340034B8
:1008A00000340034003400340034003400340034A8
:1008B0000034003400340034003400340034003498
:1008C0000034003400340034003400340034003488
:1008D0000034003400340034003400340034003478
:1008E0000034003400340034003400340034003468
:1008F0000034003400340034003400340034003458
:100900000034003400340034003400340034003447
:100910000034003400340034003400340034003437
:100920000034003400340034003400340034003427
:100930000034003400340034003400340034003417
:100940000034003400340034003400340034003407
:1009500000340034003400340034003400340034F7
:1009600000340034003400340034003400340034E7
:1009700000340034003400340034003400340034D7
:1009800000340034003400340034003400340034C7
:1009900000340034003400340034003400340034B7
:1009A00000340034003400340034003400340034A7
:1009B00004308A002608DF3E03188A0A8200903439
:1009C0000C34A2344034EA34A33460341334D034C9
:1009D00093345F3431340834E034B93492346B34B6
:1009E00044341C34F534CE34A7347F345834313495
:1009F000233416340834FA34EC34DF34D134C334BD
:100A0000B534A834A2349C34963491348B34853474
:100A10007F347A3474346E34683463345D345734DC
:100A200051344C34463440343A3439343734353424
:100A30003334313430342E342C342A3428342634B0
:100A40002534233421341F341D341C341B341A3410
:100A5000193418341734163415341434123411344C
:100A600010340F340F340E340E340D340D340C3476
:100A70000C340B340B340B340A340A340934093483
:100A80000834083407340734063406340634063490
:100A9000063405340534053405340534053405348D
:100AA0000434043404340434043404340434043486
:100AB000033403340334033403340334033403347E
:100AC0000334033403340234023402340234023473
:100AD0000234023402340234023402340234023466
:100AE000013401340134013401340134013401345E
:100AF000013401340134013401340134013401344E
:100B0000013401340134013401340134013401343D
:100B10000034003400340034003400340034003435
:100B20000034003400340034003400340034003425
:100B30000034003400340034003400340034003415
:100B40000034003400340034003400340034003405
:100B500000340034003400340034003400340034F5
:100B600000340034003400340034003400340034E5
:100B700000340034003400340034003400340034D5
:100B800000340034003400340034003400340034C5
:100B900000340034003400340034003400340034B5
:100BA00000340034003400340034003400340034A5
:100BB0000034003400340034003400340034053094
:100BC0008A002608E63E03188A0A82006934C33484
:100BD00069345434BB3491344634BB34FB34C134AF
:100BE000F634B7342B34F234BA3482344934113405
:100BF000D934A03468343034F734BF348734C73440
:100C0000073447348834C834083449348934C93403
:100C10000A344C348E34D034133455349734DA34A7
:100C20001C345E34A134E33425346834AA34EC3403
:100C30002F347134B334F63422344E347B34A73439
:100C4000D43400342D3459348534B234DE340B348A
:100C5000373464349034BD34A83494347F346B34E6
:100C6000573442342E3419340534F134DC34C8346A
:100C7000B4343D34C6344F34D8346134EA34733438
:100C8000FC3485340E3497342034A9343234BB34E8
:100C90004434CD345634DF34693448342734063490
:100CA000E534C434A3348234613441342034FF3415
:100CB000DE34BD349C347B345A343A341934F8343D
:100CC000D734B634953474345334333471345C349B
:100CD00033341534F234D934BB34A5348B347834FE
:100CE00062344D343D342B341D340C340034F13433
:100CF000E634D834CE34C234B634AE349F34923471
:100D0000853477346C3462345834513445343D344E
:100D100034342C3425341E3415340C340434FD346E
:100D2000F534EE34E834E234DC34D734D234CE3423
:100D3000CA34C634C234BF34BB34B834B534B23428
:100D4000AE34AC34A934A634A334A0349D349B34DF
:100D500098349634933491348F348C348934863477
:100D6000843481347F347D347A3479347734753403
:100D70007434723471346F346E346C346B346A345E
:100D8000693468346634653464346334623461349D
:100D900060345F345F345E345E345E345D345D34C1
:100DA0005D345C345C345B345B345B345A345A34C9
:100DB0005A345934593459345834583458345734CF
:0C0DC000573457345634563456345634E9
:02400E00C230BE
:00000001FF
